:0200000480007A
:1000000097170000938707009300100093010000EA
:100010009302F0FFB70D0080938DFDFFB70E0080B7
:10002000731000347391003473920134739302346B
:10003000739E0D34739F0E34F31F003423A02700EA
:1000400023A2470023A4670023A6C70123A8E70132
:1000500023AAF701171D0000130D4DFCB7503412F1
:100060009380806737E1BC9A130101EF73900034ED
:10007000F311013473920134F31202347313003418
:1000800023203D0023224D0023245D0023266D0004
:1000900097100000938080F9377172421301F1E6E6
:1000A000731001347310003423A0000017110000F6
:1000B000130101F8B79DFFF7938D8D8173900D3477
:1000C0007310003473100034F31200342320010045
:1000D0002322510017110000130101F6B753163205
:1000E000938383493763721413036383B75238963B
:1000F0009382422773100334F3920234F393033450
:100100007314003423205100232271002324810022
:1001100017150000130505EF97150000938585F26C
:10012000370610F01306C6F26306B5028326C50033
:100130002320D600832685002320D6008326450071
:100140002320D600832605002320D60013050501B1
:100150006FF09FFD370510F0130505F22320050011
:04016000000000009B
:10100000FFFFFFFFFFFFFFFFFFFFFFFFFFFFFFFFF0
:10101000FFFFFFFFFFFFFFFFFFFFFFFFFFFFFFFFE0
:10102000FFFFFFFFFFFFFFFFFFFFFFFFFFFFFFFFD0
:10103000FFFFFFFFFFFFFFFFFFFFFFFFFFFFFFFFC0
:040000058000000077
:00000001FF
